:10000000758150020006C200D294C2961207DBD25C
:10001000961203C5750A0A12002EE509B50A0512E3
:1000200007DB80F3F50A1200561207DB80E9209304
:100030000675090402005520920675090302005551
:1000400020910675090202005520900675090102EB
:10005000005575090022E509B4000A120394120143
:10006000221202AF22B4010D1203941201221202D5
:10007000C21200F922B4020D1203941201221202DC
:10008000D51200E422B4030D1203941201221202CD
:10009000E81200BB22B4040D1203941201221202D2
:1000A000FB1200A6222275122E7513067510037519
:1000B00011017515FFD20012030E2275122E751351
:1000C000017510037511027515F0D20012030E753B
:1000D000122E7513047510037511037515FFD200E8
:1000E00012030E2275122E75130375100375110479
:1000F0007515FFD20012030E2275122E75130175AD
:1001000010037511057515F0D20012030E75122E2D
:100110007513017510037511067515FFD2001203D2
:100120000E2275123975130175103C75110090047B
:100130000612030E7512257513017510467511010F
:1001400090043F12030E7512747513017510047537
:10015000110790076712030E7512307513017510A1
:10016000027511009003D612030E742112037774E6
:1001700002120377747F12037774221203777401DB
:10018000120377740712037774FF12035A7A2D74DF
:100190000012035ADAF9740112035A74FF12035A57
:1001A00074211203777402120377747F1203777439
:1001B000221203777402120377740712037774FF15
:1001C00012035A7A2D740012035ADAF974081203D2
:1001D0005A74FF12035A74211203777402120377C0
:1001E000747F1203777422120377740312037774F7
:1001F0000712037774FF12035A7A2D740012035A00
:10020000DAF9740012035A74FF12035A74211203AC
:10021000777402120377747F1203777422120377C4
:100220007404120377740712037774FF12035A7A67
:100230002D740012035ADAF9740112035A74FF1272
:10024000035A74211203777402120377747F120326
:1002500077742212037774051203777407120377F9
:1002600074FF12035A7A2D740012035ADAF97408D3
:1002700012035A74FF12035A742112037774021284
:100280000377747F120377742212037774061203C4
:1002900077740712037774FF12035A7A2D74801251
:1002A000035ADAF9748012035A74FF12035A227542
:1002B000123775130375103C751103900464120313
:1002C0000E2275123675130375103C7511039005D7
:1002D0000912030E2275123675130375103C751141
:1002E000039005AB12030E227512367513037510B9
:1002F0003C75110390064D12030E227512287513DA
:100300000375103C7511039006EF12030E22851140
:100310000DE50D2513F514750C007421120377E516
:1003200010120377747F1203777422120377E50D9E
:100330001203777407120377200009E49312035A1B
:10034000A3020349E51512035A050CE50CB512E8A2
:10035000050DE50DB514C0C200227F08D297C294E6
:1003600030E705D29502036AC29500D294000000DE
:1003700000C29423DFEA227F08C297C29430E705C7
:10038000D295020387C29500D29400000000C29467
:1003900023DFEA22750D00750C0074217177E50CDE
:1003A0007177747F717774227177E50D71777407B7
:1003B00071777400715A050CE50CB480F5050DE5F4
:1003C0000DB408D3229007E4750B19E4937177A359
:1003D000D50BF871942200884C2E1E0E0E0E0E0EB8
:1003E0000E0E0E0E0E0E0E0E0E0E0E0E0E0E0E0E2D
:1003F0000E0E0E0E0E0E0E0E0E0E0E0E0E0E0E0E1D
:100400000E1E2E4C88000F1008100F001C0A090A3F
:100410001C0001011F0101001F151511001F05051A
:100420000D12000000001F101010001F1515110004
:100430000708100807001F151511001F1010101FC6
:100440000204021F000E1111110E001F0204081FEA
:10045000001F0001011F0101000E1111110E001FEC
:1004600005050D12F0F03030303030303030000003
:10047000000000000000000000000000000000007C
:1004800000000000000000000000000000E0E000AC
:100490000000000000000000000000FFFF18181816
:1004A0001818181800000000FFFF0C070707FCF8D9
:1004B0000C070707FCF8000000FFFF0C0707070FF9
:1004C000FCF80007FFFF070700071FF8E000C0F86F
:1004D0003F070F0F0E0E0E0E0E0E0E0E0000000F39
:1004E0000F000000000F0F000000000F0F000000C1
:1004F000FFFF030E0E0E0F03010000030F0E0E0090
:1005000000C0C0FF7F0F00000000C0E0603030304E
:10051000303070E0C08000000000C0F0703030303B
:1005200030303030300000000000C0F038181818AB
:1005300038F0C000000000C0F038080000000003E0
:1005400003000000000080C0E0703F0F0000003892
:100550003F1F180C0C0C0C0C1838F0C000000000E9
:10056000071F38303030381F87E0703C0FC3E06021
:100570006060E0C000C0F0F8DCCCC6C3C3C1C0C03E
:10058000C0C00000000C3C7060C0C0C0C0E060781B
:100590001F0F000000000000000080E0781E07012F
:1005A00000001F7FE0C0C0C0E07F1F00C0F07030BF
:1005B00030303030303030000000000080E06030FB
:1005C0003030303060E0800000000000C0F03818AB
:1005D000181838F0C000000000C0F0380800000013
:1005E00000383F1F180C0C0C0C0C1838F0C0000021
:1005F00000FEFF010000000000000001FFFE0000FF
:100600000000071F38303030381F87E0703C0FC3C0
:10061000E0606060E0C0000C3C7060C0C0C0C0E042
:1006200060781F0F000000071F7860C0C0C0C0C006
:1006300060781F07000000000000000080E0781EC6
:10064000070100001F7FE0C0C0C0E07F1F303030D6
:10065000303030303030B0F0F03000000000C0F00A
:100660007030303030303030300000000000C0F0EA
:100670003818181838F0C000000000C0F038080022
:10068000000000000000000080E0781E070100006C
:10069000000000383F1F180C0C0C0C0C1838F0C070
:1006A00000000000071F38303030181F87E0703C12
:1006B0000FC3E0606060E0C000000000F0FE1F03B8
:1006C0000000000000000000000C3C7060C0C0C0D2
:1006D000C0E060781F0F000000000000000080E014
:1006E000781E070100001F7FE0C0C0C0E07F1FF040
:1006F000F03030303030303030303000000000002A
:10070000000000000000000000000000000000F0F9
:10071000F000000000F0F0FFFF606060606060606B
:1007200060600000000000FEFE000000000000000D
:1007300000FEFE00000000FFFF00000000FFFFFFC2
:10074000FF00000000000000000000000000001F8B
:100750007F60C0C0C0C0C06030FFFF00000000FF6D
:10076000FF00000000FFFF1C60180418601C000060
:100770001C60180418601C00001C60180418601C21
:10078000004000007E080870000038444438000033
:100790007E48483000007E484830000418E01804C5
:1007A00000FC2424180000FC040038444438008075
:1007B0007D000038545458000038444400043F443D
:1007C00000485424000040000038444400003844ED
:1007D000443800007C0404780404787DFF7CFFDC4E
:1007E000FEDDFA22AED580A83FD300408D14200252
:0D07F000A1C8DA1281CFD9F1DB40A4A6AF79
:00000001FF
